:020000040000FA
:060000000219FD0200C818
:03000B0002008D63
:03002B000200923E
:03005B000202CBD3
:030073000200B5D3
:100080000406080C10182030406080A0C0C28D0506
:100090004032C0D0C0E0C2CF0541E5646009E563ED
:1000A000600575630001B0756301E52360021523E7
:1000B000D0E0D0D032C2AF53E67F7592FA7593FF8D
:1000C000C22053917FD2AF32C2AF53E6EFC0D0C04F
:1000D000E0C0F0D2D3D2AF5388EFA88AA98CAA404F
:1000E000308D010A758A00758C00754000438810B8
:1000F000E564700AC3E833F8E933F9EA33FA3033D8
:100100001FE8C4540FFAE9C454F04AFAC3132AFA98
:10011000C3E833F8E933F9E82AFAE93406FB217336
:1001200030320FC3E833E933FAE82AFAE93400FB46
:100130002173303115E875F056A4AAF0E975F05630
:10014000A42AFAC5F03400FB2173C3EA13FAE913B9
:10015000F9E813F8E875F056A4AAF0E975F056A48A
:100160002AFAC5F03400C313FBEA13FAC3EB13FBFE
:10017000EA13FAC3EB94125006C3EB9406501A0527
:1001800022E52270021522C3E522940A500241BEE4
:100190007552007A007B00418CE522600215223006
:1001A00035067C007D0821B3AC31AD32303A04AC69
:1001B00033AD34C3EA9CFAEB9DFB9208AE5EAF5FB1
:1001C000303A425007203409D23421D1303402C2AF
:1001D00034303404AE60AF61203902B234C3EA3344
:1001E000FAEB33FBA208500AEAF42401FAEBF434E8
:1001F00000FBC3EA9450FAEB9400FB501478007AA9
:10020000007B004111A208500878007A007B004171
:1002100070E5255403601B202A18E55B33F9EB7069
:1002200007C3E99A4002E9FAE53CC4332AFAEB3401
:1002300000FBEA8EF0A4F9AAF0EB8EF0A42AFAC52E
:10024000F03400FBC3EB13FDEA13F8C3ED13FDE834
:1002500013F80FEF146004C3E833F8C3E933EA334B
:10026000FAEB33FBDFEDEB30E30678FF7AFF7B0739
:100270008852D230C3E559FC955A4002AC5AC3ECBF
:1002800095525008EC75F008A4FAABF0EAF4F8EBDC
:10029000F45407F9C3E89450FAE99400FB50047A47
:1002A000007B00885489558A568B5775230AD0F0F5
:1002B000D0E0D0D053F7DF43F74043E61032752348
:1002C0000AD0F0D0E0D0D043E61032C2AF53A8FE3F
:1002D000C0D0C0E0D2D3A8F9E55830E20AE5FA2050
:1002E000E24220E13F41EFE5FA30E23820E135C358
:1002F000E55513F8E55413F5FB88FCC3E55713F8EF
:10030000E55613F5E988EA85555853F7BFC3E5521A
:10031000940140057553006124E5532401F55350C1
:10032000037553FF53F7DFD0E0D0D043A801D2AF1D
:10033000327901801479038010790A800C791E804B
:10034000087964800479C880007817E4D5E0FDD886
:10035000FAD9F6227A147B7880127A107B8C800C82
:100360007A0D7BB480067A0B7BC88000E562D5E00D
:1003700001227902E4C291D5E0FDD290D5E0FDC220
:1003800090D5E0FDD291D5E0FDE920E002D28630A3
:10039000E002D292E562D5E0FDE920E002C28630BB
:1003A000E002C2927496D5E0FDD9C9EAF8D5E0FD25
:1003B000D8FBDBB8C2912278FF20282879A1E7601A
:1003C00023E548601F74FF8548F084853FF030299D
:1003D0000375F005A4F8C5F0600278FFC3E8955BEB
:1003E0005002A85B885A22C3E54794A0E5489400D0
:1003F000E55A50031461F8046002F55A2275E8903A
:1004000022055CC3E55C9408405330EDF4A8BDA917
:10041000BE755C00E9FA79A0E76041EA7006E55D27
:100420006018800CC3E8955D600EE55D5005600ABC
:100430001480070460FA8002E55DF55DC3956740AE
:100440001B7559C0C394044013755980C39404406C
:100450000B755940C39404400375590022E5592493
:1004600010500274FFF55922743279A687F0A4C5A2
:10047000F0A2F733F8C3E895594002A859885B22E7
:100480007547007548F022C2AF75C800A8CCA9CD49
:10049000AA4130CF010A75C804D2AFC3EA13FAE902
:1004A00013F9E813F8AB42AC4388428943C3E89B95
:1004B000F8E99C20280A547FF9302C02A1A481FE7F
:1004C000AD448A44F9EA9D547FFA600478FF79FFCD
:1004D000AE45AF468B458C46A842A943C3E89EF87B
:1004E000E99FF9C3E54813FBE54713FAE82AF54706
:1004F000E93BF54850067547FF7548FFA14BAA47F1
:10050000AB48AC47AD487E047F02C3EB9404400D7A
:100510001E1FC3EB940840052029021E1FC3ED13C4
:10052000FDEC13FCDEF7C3EA9CFAEB9DFBEF6009E0
:10053000C3E913F9E813F8DFF7EA28FAEB39FB8A85
:10054000478B4850067BFF8B478B48C3EB94025088
:1005500002D22C3028047F03A1767892E6FFC3E50F
:100560003D948240110FC3E53D94A040010FC3EFBD
:10057000940640027F057E02E548C4540FF9E54821
:10058000C454F0F8E547C4540F28F8C3E89EFAE9CC
:100590009400FB4009C3EA9401EB940050047A01F3
:1005A000E4FBA1F0AA47AB48EBC4FEEAC4540F4EEB
:1005B000FCC3EA9CFAEB9400FBC3E813C313F8EA0C
:1005C00028FAEB3400FB8A478B48C3EB94024002C5
:1005D000C22C7802EBC4FE7B00EAC4540F4EFAC36F
:1005E000EA98FA4005C3940150027A017892E6FF36
:1005F000302002A1F0854E92854F93D22043E680B1
:10060000C3E49AF8E49BF9C3E833F8E933F9302CF2
:1006100002C182E8FAE9FBD3E913FDE813FC884E36
:10062000894FC3EF94036037EF20E00CE82CF8E922
:100630003DF9ECFAEDFB8013E828F8E939F9C3E855
:100640002401F8E93400F97AFF7BFFC3EF940340FB
:100650000E8A508B51884A894B8C4C8D4DC1B6887F
:100660005089518A4A8B4B8C4C8D4D3028127550D5
:10067000F07551FF754CF0754DFF754EF0754FFFDD
:10068000C1B6E8FAD3E813FC884EC3EF94036020A8
:10069000EF20E007E82CF8ECFAC1A2E8282401F8E2
:1006A0007AFFC3EF940340088A50884A8C4CC1B645
:1006B00088508A4A8C4C302002C1B6753A02D2204A
:1006C00043E680E5255403602DA847A948C3E913F4
:1006D000F9E813F8302804E92440F9C2AF53E67F63
:1006E000759100C3E498F594E499F595759104D259
:1006F0002043E680D2AF22D2217549007520003018
:100700002B03752040800ED22175490075204030A2
:100710002B0375200078017901202C20E525540356
:100720006002C2217914E548C313700104F8C39430
:100730001440027814302804781B791BC3E833F87E
:10074000C3E933F9202010E549600C302803D53A7D
:1007500004D223E1CBD1BE0549E59B5440B520022C
:10076000E1B530280908C3E899400118E144202187
:100770000A08C3E8994002E115E144C221C2AF531F
:10078000E67F759100302C127594007595F0759187
:1007900004D22043E680D2AFE115E5487EFFC333A3
:1007A0004009C3334005C3334001FEC3E49E759442
:1007B00000F595E18EC3E53994015002E115302131
:1007C00002E115D802E1C9E144C223C2AF53E67F7A
:1007D000759100855094855195759104854A92854F
:1007E0004B93D22043E680D2AFE525540360072027
:1007F00029020539801030230D202B0A20210715EE
:10080000811581020F2E2278003021027801E53D0A
:1008100075F007A4F9E5F028F5F0E9A2F013A2F1CC
:1008200013A2F213F53DC394785003753D78C3E5E8
:100830003D953E400ED222C286C290C29275D4FF30
:1008400075D50F3020020143854C92854D93D220FF
:1008500043E68022203813C2AFC291D28775D4FFFD
:1008600075D503D2AF759F42214CC2AFC291D293CE
:1008700075D43F75D50FD2AF759F42214C203814E7
:10088000C2AFC29275D4FF75D50CD287D2AF759F17
:100890005202094CC2AFC28675D4FF75D50CD293F3
:1008A000D2AF759F3202094C203813C2AFC287D233
:1008B0009375D4FF75D50CD2AF759F32214CC2AF62
:1008C000C293D28775D4FF75D50CD2AF759F528075
:1008D0007B203814C2AFC29075D43F75D50FD29328
:1008E000D2AF759F4202094CC2AFC29075D4FF755A
:1008F000D503D287D2AF759F4202094C203813C26C
:10090000AFC293D29175D43F75D50FD2AF759F52B8
:10091000803AC2AFC287D29175D4FF75D503D2AFEA
:10092000759F328027203813C2AFC28675D4FF75F9
:10093000D503D291D2AF759F328011C2AFC29275EA
:10094000D43F75D50FD291D2AF759F52C22222C229
:1009500086C290C292C287C291C29375D4FF75D5E8
:100960000F22788076FF0876FF0876FF0876FF086A
:1009700076FF0876FF0876090876FF087601788CFE
:1009800076010876FF0876FF0876FF0876FF08767E
:10099000FF0876030876FF0876FF0876FF087625BD
:1009A0000876D00876280876500876040876FF087E
:1009B00076020876FF08767A0876FF0876070876CA
:1009C000010876FF0876FF08760008760022FA759F
:1009D000F00CA4ABF0EAC333F8740133F9E8C33385
:1009E000F8E933F9E8C32BF8E93400F9E8C333F840
:1009F000E933F9227888E6C39403D23A5002C23A26
:100A0000C238E630E102D238A23892397886E6144C
:100A10009000809378A6F67886E6F53FC39402505E
:100A200003753F02789CE6753EFFB40203753EA055
:100A3000B40303753E8278A0E6F8600674282409A2
:100A4000D8FCF5677896E631CE88318932789EE613
:100A500031CE883389347897E631CE88358936317E
:100A60004F223035117A007B007CFF7D007E0051E3
:100A7000C98B5F8A5E22303A227896E6FA7B00784C
:100A80009EE6FC7D00C3EA33FAEB33FBC3EC33FC98
:100A9000ED33FD7E0A51C98B618A607896303A0247
:100AA000789EE6FA7B007897E6FC7D007E00303A7F
:100AB00010C3EA33FAEB33FBC3EC33FCED33FD7EBA
:100AC0000A51C98B5F8A5E2222C3EC9EFCED940022
:100AD000FDC3EC9AFCED9BFDC3EC9423ED94005018
:100AE000047C237D00C3EC94FFED940140047CFF63
:100AF0007D017BFF0B7A000AEA7009C3EC33FCED41
:100B000033FD41F4EC8AF0A4AEF0ED8AF0A42E940B
:100B10007C40E4EAF460DD22D235516212033D12DA
:100B2000033D7A007B007C10120335E5522AFA74EB
:100B3000003BFBDCF37C04C3EB13FBEA13FADCF7AA
:100B4000FFEB60027FFFC23551622278A5E6F954BF
:100B5000037000E9540C7000E954307000E954C08F
:100B60007000227565007566007597DE7597AD7526
:100B700081C043FF8075EF0675A900314F75803F36
:100B800075F1C375A4C075803F75D4FF759000756D
:100B9000F20F75A50F75900075D50F75A60175E359
:100BA0004075E202314FE4F8F6D8FD3162F16F781A
:100BB000988662753001C2AF1203451203541203C6
:100BC0003D12035A12033D12036012033D714BC2E2
:100BD000AF75650075660078FA79FA308007D9FB41
:100BE000D8F7021C0031F4516278988662314F7553
:100BF000A91375A71075C10075A70075640075E489
:100C000000758811758E0475890975C8047591047D
:100C100075D84075D90875F782759E03759602756B
:100C2000DA4275DB4275A82375E69075F310759B63
:100C300080759D0075D10C75BCB975BB1075E880C9
:100C400075B201120331D2AF753C00C230120345B8
:100C5000C231752200120341C3E522940A4024D216
:100C600031C232752200120341C3E522940A4013B7
:100C7000D232C233752200120341C3E522940A40E6
:100C800002D233120335203003020BCFC2AF12035E
:100C900054120354120354D2AF120345303A02A146
:100CA00041120335788CE6C394015002A141E5302E
:100CB000C394015002A1417565A57566F17F02D20A
:100CC000355162120341C2AFC2355162C3E552943D
:100CD0007FD2AF406C120331C2AF120366D2AFDFD6
:100CE000DE7118C3EF7897F61203451210577F0A8A
:100CF000D2355162120341C2AFC2355162C3E552CF
:100D0000947FD2AF50E8120331C2AF1203541203E2
:100D100039120354D2AFDFD87118EF24037896F656
:100D2000F87997E7C394234003985006E824237882
:100D300097F6120345F1A912108612034151626120
:100D4000CF7565007566001203417801303A02786C
:100D500005C3E552984002819CC2AF12036612039C
:100D600066120366D2AF120345753000E4F537F51D
:100D7000380537E537F4703E0538789AE678191467
:100D80006012783214600D787D14600878FA14606F
:100D900003753800C3E53898401C314F12033115F4
:100DA0003875370078998662C2AF120366D2AF7881
:100DB000988662120341120339E523700261CF78ED
:100DC00001C3E5529840AA120341E5237003020BC8
:100DD000CFC2AF314FE4D2AFE4F55CF524F525F591
:100DE0003D755C081203311203FD30EDFDA8BDA96D
:100DF000BEE97001F8885D120401755C08C2AF7528
:100E000059FF120468855B59855B5AD2AF75A710EC
:100E100075C13075A70075A903756401303A07C222
:100E200038303402D238D22875390011FC312512FD
:100E300004801204871204801204871204801207AF
:100E400007110711541204871206F7202C0312030E
:100E5000B7302C031203E71107117D120487120724
:100E600007110711A81204871206F7110711D112F2
:100E70000487120707110711FC1204871203FD12E1
:100E800006F711073125120401120487302827853F
:100E90005B5979187A0CC3E53999400EC228D229DA
:100EA0008A3B855B59855B5A800CC3E552940140AF
:100EB00003020E3EE13630291C202B19E53B14704D
:100EC00006C229D22AC13EF53BC3E5529401400334
:100ED000020E3E8061753C0078FA79A4E7600278E2
:100EE00003C3E55398504FE523604B303A17203841
:100EF00005203407800F303402800A202B07D22BC4
:100F0000855B59C16878F0302B05855B597820C323
:100F1000E548985003020E3E302B1BC22BC23830DE
:100F20003402D238D229753B12855B59C13E053C4B
:100F3000E5526002E139753C00C2AF314F752400C3
:100F400075250075A91375A71075C10075A70075E3
:100F50006400D2AF120341314F78A4E66006D28715
:100F6000D291D293C3E53C9404400261CFA16C902E
:100F70001A0D7820F1E6E520B4550AA3F1E6E52044
:100F8000B4AA0280063162F1A9801D901A0378800C
:100F90007B0AF1E6A308DBFA901A0F788C7B1AF132
:100FA000E6A308DBFA901A2922C2AF12102B121006
:100FB00006901A007410F1EBA37403F1EBA37421F3
:100FC000F1EB901A0378807B0AF1EAA308DBFA9030
:100FD0001A0F788C7B1AF1EAA308DBFA12103F1281
:100FE000101A901A2922E493F622E6438F01538FB8
:100FF000FDFFC3E583941C400122EF8565B785663C
:10100000B7F0538FFE22438F02438F018565B7856A
:1010100066B7901A0DF0538FFC22901A0D7455127A
:101020000FEB901A0E74AA120FEB227A3079D07857
:1010300020901A40120FE6E520F709A3DAF6227A8B
:101040003079D0901A40E7120FEB09A3DAF8227C2E
:1010500005120345DCFB22C2AF12035412035A12DD
:10106000036012036612033912035412035A120367
:101070006012036612033912035412035A120360FA
:10108000120366D2AF22C2AF1203661203601203CC
:101090005A12035412033912036612036012035AE0
:1010A00012035412033912036612036012035A1218
:0510B0000354D2AF2241
:1019FD00020B63100321FFFFFFFFFFFF09FF01FF34
:101A0D0055AA01FFFFFFFFFF03FFFFFF25D0285061
:0D1A1D0004FF02FF7AFF0701FFFF0000FF3A
:101A400023435F485F3430232020202020202020A3
:101A500023424C48454C492445464D3842323123B7
:101A60002020202020202020202020202020202076
:101C0000C2AFC2D37597DE7597AD7581C075A90057
:101C100043FF80752438752503B1DB7529A5752A26
:101C2000F143F10153A4FED28075D4FF75E3407DEA
:101C3000FA780379E67C10752200752300901DE880
:101C40007B06752498752501308002814820800824
:101C5000D8FBD9F9DCF781BA308008D8FBD9F9DC98
:101C6000F781BAB19BE493A3C39A6004DDC381BA40
:101C7000DBDBB18D600281317B08E493FAA3B16EA6
:101C8000DBF87A30B16E752200752300B18DEAFC65
:101C9000EBFDC3ED94FE400EB18D8A278B28ED300D
:101CA000E0048A828B83B18D7AC270D8C3ED94FE32
:101CB000601950CEBD0029EC600F7520007521FF22
:101CC000752900752A000200008100A827A92808AC
:101CD00009D804D90281DDB191EAF281D10D81A642
:101CE000C3ED94035051EDA2E092007AC5C3E582A2
:101CF0009400E583941C508C200010438F02438F86
:101D0000018529B7852AB7F0300027A827A9280818
:101D100009438F01538FFDD804D902A132C3E58353
:101D2000941C4003A3A117E28529B7852AB7F0A325
:101D3000A117538FFC81827AC1BD030CE493A3FAEF
:101D4000B152DCF8B14A81828184AA22AB23B16E00
:101D5000EBFAEA6222752608C3E52313F523E52290
:101D600013F52250066323A0632201D526EAB1DBD6
:101D7000B1DB75260AEAF4200102D280300102C2EA
:101D800080B1DBC3134002C201D526EB22B191EA38
:101D9000FB208002A191308002A196752608AE2416
:101DA000AF25C3EF13FFEE13FEB1DFB1DBC3EA13C0
:101DB0003080024480FA30E703632201C3E5231335
:101DC000F523E52213F52250066323A0632201D5F3
:101DD00026D9E52265236523F52222AE24AF250E00
:101DE0000FDEFEDFFCD20122424C48656C693437BD
:061DF0003163E8B20601B8
:00000001FF
